:1000000092C020C8ABC0AAC0A9C0A8C0A7C0A6C043
:10001000A5C0B7C9A3C0A2C0A1C0A0C09FC09EC0B8
:100020009DC09CC09BC000000001010203030405A9
:100030000506070708090A0A0B0C0D0D0E0F101113
:10004000121213141516171818191A1B1C1D1E1F2F
:1000500020212122232425262728292A2B2C2D2E36
:100060002F303132333435363738393A3B3C3D3E28
:100070003F4041424345464748494A4B4C4D4E4F0D
:100080005051535455565758595A5B5D5E5F6061E5
:10009000626364666768696A6B6C6E6F70717273B5
:1000A00075767778797A7C7D7E7F8081838485867A
:1000B00087898A8B8C8D8F90919294959697989A38
:1000C0009B9C9D9FA0A1A2A4A5A6A7A9AAABACAEEC
:1000D000AFB0B1B3B4B5B6B8B9BABBBDBEBFC1C29B
:1000E000C3C4C6C7C8CACBCCCDCFD0D1D3D4D5D743
:1000F000D8D9DADCDDDEE0E1E2E4E5E6E8E9EAECE5
:10010000EDEEF0F1F2F4F5F6F8F9FAFCFDFEFFFF82
:10011000FFFFFFFFFFFFFFFFFFFFFFFFFFFFFFFFEF
:10012000FFFFFFFFFFFF11241FBECFE5D4E0DEBFBE
:10013000CDBF11E0A0E6B0E0E0E5F8E102C0059037
:100140000D92A837B107D9F714E0A8E7B1E001C0D4
:100150001D92AB34B107E1F707D578CB51CF482FCB
:1001600090E820E030E0FB01E20FF31F892F8423A9
:10017000808396952F5F3F4F28303105A1F7089572
:10018000982F80914602882331F028E431E740E03F
:1001900050E0ACE005C028EA31E640E050E0A0E0E5
:1001A0006058E62FFF27E7FDF095892F992787FDF7
:1001B0009095E81BF90BAA23F9F01E161F0654F4BC
:1001C0008A2F992787FD9095E817F9079CF0E81B7F
:1001D000F90B12C0309781F06A2F772767FD709571
:1001E00088279927861B970B8E179F071CF0E60F11
:1001F000F71F02C0E0E0F0E0BF01882777FD80959F
:10020000982F8EDA20E03DE740E050E0A8DA8FEF4B
:10021000223838071CF421E83FEF05C020383105AB
:1002200014F02FE730E0C90108952F923F924F92CA
:100230005F926F927F928F929F92AF92BF92CF9276
:10024000DF92EF92FF920F931F93DF93CF93CDB77F
:10025000DEB72A970FB6F894DEBF0FBECDBF6C0194
:100260007A876987FC0186818071FB018183F601B1
:1002700086818870E985FA858583F6018681807894
:10028000E985FA858187F60186818170E985FA859D
:100290008587F60186818072E985FA85818BF60172
:1002A00086818074E985FA85858B7896F887EF8357
:1002B000F60183818058EF81F8858183F60183817F
:1002C0008058E985FA85858FB096FE83ED83F60127
:1002D00082818058ED81FE818183F6018281805880
:1002E000E985FA8585A3F60187818170E985FA851C
:1002F00081A7F60187818270E985FA8585A7F601D5
:1003000087818870E985FA8581ABF60187818470E1
:10031000E985FA8585ABF896FC83EB8389859A8518
:10032000CC969A83898380917801F601608128DFD9
:100330001C014C01AA2497FCA094BA2C809179014D
:10034000F60161811DDF2C01662457FC6094762C38
:1003500097FF03C0909581959F4F682F70E080E0D4
:1003600090E0A5019401DCD920E032E040E050E0CB
:10037000F6D979018A01E80CF91C0A1D1B1DC1017F
:1003800037FE03C0909581959F4F682F70E080E005
:1003900090E0A3019201C4D920E032E040E050E0B7
:1003A000DED9240D351D461D571DF2E8EF16FFEF6F
:1003B000FF06FFEF0F07FFEF1F074CF491E8E92E50
:1003C0009FEFF92E9FEF092F9FEF192F0BC080E8A9
:1003D000E816F104010511052CF08FE7E82EF12C49
:1003E000012D112D22389FEF39079FEF49079FEF0D
:1003F00059072CF421E83FEF4FEF5FEF09C0203899
:1004000031054105510524F02FE730E040E050E090
:10041000EB81FC81E182E981FA81218389859A85DA
:10042000805C9F4F9A878987F60186818470E98571
:10043000FA8581833496FA87E987F601868182708E
:10044000E985FA8581833496FA87E987E981FA811B
:100450008181E985FA8581833496FA87E987E98184
:10046000FA818181E985FA8581833496FA87E98763
:10047000EB81FC818181E985FA8581833496FA8755
:10048000E987EB81FC818181E985FA858183349656
:10049000FA87E987F60184818058E985FA858183A6
:1004A0003496FA87E987F60185818058E985FA85CF
:1004B00081833496FA87E987ED81FE818181E98520
:1004C000FA8581833496FA87E987EF81F8858181FF
:1004D000E985FA8581832A960FB6F894DEBF0FBEB0
:1004E000CDBFCF91DF911F910F91FF90EF90DF90E3
:1004F000CF90BF90AF909F908F907F906F905F90C4
:100500004F903F902F900895CF93DF93C0E0DAEFA4
:10051000CE010197F1F7E091FC01F091FD01048417
:10052000F585E02D80E00995E091FC01F091FD0159
:100530000684F785E02D0995882351F3E091FC01AD
:10054000F091FD010088F189E02D8EEF91E0099591
:100550008EEF91E06EEA70E068DE20E030E080919E
:10056000AF00882311F021E030E08091B3008111C9
:1005700022608091EF00811124608091F30081114D
:1005800028608091B700811120618091BF008111A6
:1005900020628091C300811120648091D700811175
:1005A00020688091DB00811131608091DF00811132
:1005B00032608091E300811134608091BB00811131
:1005C0003860E0917C01F0917D01E227F32741E062
:1005D00050E060E070E0CA018E239F23892B69F010
:1005E000CA0182239323892B41F030937D0120930C
:1005F0007C01CA01DF91CF910895440F551F6F5FB1
:100600007F4F6C30710539F730937D0120937C0169
:100610007FCFDF92EF92FF920F931F93CF93DF93E1
:100620007B01D42E052F8032910519F0EB0110E8E3
:100630000EC0FB0180819181FFEF8F3F9F0709F47E
:1006400051C00196FB019183808349C05DDF8830F2
:100650009105D1F1893091054CF48230910561F119
:100660008430910569F1019789F723C080329105A3
:1006700079F1F8E080309F07A9F1409739F71038F9
:1006800041F0188319828D2D902F9C01E90110E80B
:10069000DDCFF70180819181FFEF8F3F9F0711F13F
:1006A0000196F701918380838D2D902F9C01E901A4
:1006B000CDCF110F110FCACF110F110F1F5FC6CF72
:1006C000110F110F1E5FC2CF110F110F1D5FBECF93
:1006D000CE15DF0539F0103811F01883198220E0AB
:1006E00030E002C02FEF3FEFC901DF91CF911F91A2
:1006F0000F91FF90EF90DF900895CF93DF93DC018F
:10070000EB0120E011969C91119713968C91139711
:10071000981321E02883FD01349620E091818381A4
:10072000981321E02983FD01389620E0918183818F
:10073000981321E02A83FD013C9620E0918183817A
:10074000981321E02B83FD01B89620E091818381ED
:10075000981321E02C83FD01BC9620E091818381D8
:10076000981321E02D83FD01F09620E09181838193
:10077000981321E02E83FD01F49620E0918183817E
:10078000981321E02F8318861986FD01709620E0CA
:1007900091818381981321E02A87FD01749620E0DE
:1007A00091818381981321E02B87FD01789620E0C9
:1007B00091818381981321E02C87FD017C9620E0B4
:1007C00091818381981321E02D87FD01B09620E06F
:1007D00091818381981321E02E87FD01B49620E05A
:1007E00091818381981321E02F87D9963C91D997E5
:1007F000DD962C91DD97FD01E05CFF4F91818381B7
:10080000981709F4922FFD01EC5BFF4F5181838112
:10081000581709F4592FFD01E85BFF4F918183813F
:10082000981709F4932FFD01E45BFF4F4181838109
:10083000481709F4492FFE01709690E89E01285E42
:100840003F4F892F842381939695E217F307C9F7C9
:10085000252F209590E8BE01605E7F4F892F82236F
:1008600081939695E617F707C9F7DF91CF91089521
:1008700090E080914602882309F491E0909346022B
:10088000AED50895A6E0B2E0E0E6F0E028E30190FE
:100890000D922150E1F79C01215030402430310568
:1008A000C0F488E390E0289FF001299FF00D389F65
:1008B000F00D1124E95BFD4F80818F3F19F42FEF7C
:1008C0003FEF09C0A6E0B2E088E301900D928150AD
:1008D000E1F720E030E0C90108959C01215030404B
:1008E0002430310598F488E390E0289FF001299F97
:1008F000F00D389FF00D1124E95BFD4FA6E0B2E04A
:1009000088E30D9001928150E1F769D5089581E067
:1009100090E015D5F9DD21E080309207E1F021E08B
:10092000813092073CF48031910519F180389105AE
:1009300061F40EC024E080309207A1F028E08030FE
:10094000920799F08050924049F02FEF3FEF14C08A
:1009500081E090E005C082E090E002C083E090E09A
:10096000BCDF08C084E090E0FBCF80E090E08ADF4D
:1009700001C07EDF20E030E0C9010895BF92CF9230
:10098000DF92EF92FF920F931F93DF93CF9300D0EC
:1009900000D0CDB7DEB78FEF9FEF9A8389839C831A
:1009A0008B83BFB6F894BCD485E090E0C8D400E057
:1009B0001AEFE091FC01F091FD010484F585E02D32
:1009C00080E00995E091FC01F091FD010088F1893A
:1009D000E02D8EEF91E009958EEF91E06EEA70E0E8
:1009E00024DC8091BB00882321F0C8010197F1F736
:1009F000E0CF01E010E0B3E0CB2ED12CCC0EDD1E19
:100A00007E010894E11CF11C7FDD9C018032910580
:100A100009F443C08132910594F48430910509F4BE
:100A20003CC08530910524F40197029768F735C0E2
:100A30008830910591F18031910531F72EC081E028
:100A400020303807D9F081E0213038073CF42034D9
:100A50003105F1F020383105B9F60DC084E02030C1
:100A6000380791F088E02030380709F44CC0205056
:100A7000324051F606C081E090E008C082E090E08C
:100A800005C083E090E002C084E090E0FBDE01C09E
:100A90003EDF8F5F9F4FB9F523C0C901B701A601A3
:100AA000B8DD8F5F9F4FE1F089819A818F5F9F4F03
:100AB000B9F08B819C818F5F9F4F91F0012B19F0D2
:100AC00080E090E0DFDE69817A814B815C8186E0A5
:100AD00092E090D381E090E032D400E010E094CF37
:100AE00083E090E02CD481E090E01DD488E59BE188
:100AF00020E931E0F9013197F1F70197D9F780E06A
:100B000090E011D403C083E090E019D4A2D4BFBE1A
:100B10000F900F900F900F90CF91DF911F910F9139
:100B2000FF90EF90DF90CF90BF900895FC018585F6
:100B3000882391F04AD4882399F080917A0190918A
:100B40007B01019690937B0180937A01069744F094
:100B500015DF21E030E006C010927B0110927A018F
:100B600020E030E0C90108950F931F93CF93DF93E6
:100B7000E9D09093FD018093FC0111BA82B38B6F91
:100B800082BB889A14BA8FEF85BB85B7886085BF12
:100B900085B78B7F85BF8BB780648BBF2FEA31E031
:100BA000C90160E070E040E250E023D62FEC31E074
:100BB000C90160E070E040E250E01BD695E0909300
:100BC000EF011092F00182E08093F1019093F20125
:100BD0001092F3011092F4017894A2D381E090E096
:100BE000AED305D4892B19F082E090E0A8D3809190
:100BF000450290E047DEE0D3E091FC01F091FD0179
:100C00000284F385E02D0995909A88E893E120E924
:100C100031E0F9013197F1F70197D9F704C0CE011E
:100C20000197F1F702C0C0E0DAEFE091FC01F0912A
:100C3000FD010484F585E02D81E00995882379F78D
:100C4000E091FC01F091FD010088F189E02D8EEF2B
:100C500091E00995CE010197F1F78091FE0180584E
:100C6000809378018091FF018058809379018EEF05
:100C700091E06EEA70E0D9DA8091BB00882319F028
:100C80008EEA90E07BDE9098E4D300E08091F5015D
:100C9000882319F01092F501EAD33CD48823B1F3EC
:100CA000909A82D3E091FC01F091FD010484F585D6
:100CB000E02D80E00995182F7BD39098112339F00F
:100CC0000F5F05312CF081E090E039D3AECF00E02A
:100CD000E091FC01F091FD010684F785E02D099576
:100CE000882361F1909AE091FC01F091FD01008868
:100CF000F189E02D8EEF91E009958EEF91E06EEA9B
:100D000070E093DA86E092E06EEA70E04AE151E04A
:100D1000A8D28091F601882319F46FEC71E002C02B
:100D20006FEA71E08AE191E0E8DC8091F60190E001
:100D3000882309F491E09093F60190988EEA90E070
:100D4000F5DEA4CF88E990E00895009741F0DC013A
:100D5000EEE7F1E088E001900D928150E1F7A6E81E
:100D6000B1E0EEE7F1E088E001900D928150E1F70B
:100D700008958091AC009091AD00892B31F01092D4
:100D8000AD001092AC0081E008958EE791E066E836
:100D900071E048E050E020D50895DF93CF93CDB7C0
:100DA000DEB728970FB6F894DEBF0FBECDBFFE01A9
:100DB000319688E0DF011D928A95E9F7498120E0AC
:100DC00030E060E870E0F901E95AFC4F8081882347
:100DD00039F0CB01022E02C0959587950A94E2F76F
:100DE000482B2F5F3F4F2830310569F749834A81EF
:100DF00020E030E060E870E0F901E15AFC4F8081CA
:100E0000882339F0CB01022E02C0959587950A946C
:100E1000E2F7482B2F5F3F4F2830310569F74095A7
:100E20004A834B8120E030E060E870E0F901E95945
:100E3000FC4F8081882339F0CB01022E02C09595AA
:100E400087950A94E2F7482B2F5F3F4F28303105F2
:100E500069F74B834C8120E030E060E870E0F901F5
:100E6000E159FC4F8081882311F080E007C0CB015D
:100E7000022E02C0959587950A94E2F7482B2F5FC2
:100E80003F4F2830310559F74C834D8120E030E049
:100E900060E870E0F901E958FC4F8081882339F05F
:100EA000CB01022E02C0959587950A94E2F7482B54
:100EB0002F5F3F4F2830310569F740954D834E81B4
:100EC00020E030E060E870E0F901E158FC4F8081FB
:100ED000882339F0CB01022E02C0959587950A949C
:100EE000E2F7482B2F5F3F4F2830310569F74095D7
:100EF0004E834F8120E030E061E070E0F901E65B75
:100F0000FC4F8081882339F0CB01022E02C0880F6C
:100F1000991F0A94E2F7482B2F5F3F4F2530310588
:100F200069F720E030E060E270E0F901E05BFC4F3F
:100F30008081882339F0CB01022E02C0880F991FCF
:100F40000A94E2F7482B2F5F3F4F2330310569F7B2
:100F50004F83488520E030E061E070E0F901ED5A10
:100F6000FC4F8081882339F0CB01022E02C0880F0C
:100F7000991F0A94E2F7482B2F5F3F4F2430310529
:100F800069F7898180937E018A8180937F018B81BB
:100F9000809380018C81809381018D818093820177
:100FA0008E81809383018F8180938401409385019A
:100FB00028960FB6F894DEBF0FBECDBFCF91DF915C
:100FC0000895DF93CF93CDB7DEB729970FB6F89486
:100FD000DEBF0FBECDBF1982CE01019661E070E089
:100FE000B1D2883199F488EC90E00197F1F780E470
:100FF0008A8383E08B831C82CE01029663E070E0DB
:10100000A1D2803419F4C9DE80E001C081E02996C4
:101010000FB6F894DEBF0FBECDBFCF91DF9108951C
:1010200081E0CFDF90E0882309F491E0892F0895D3
:101030008FB7F894B99AC198A398AB988FBF81E005
:10104000C0DF08951F921FB6EF93FF934F930F9346
:101050001F937F93EEE8F1E009E00EC016E01A95C9
:10106000D1F040B34470D9F7000000000000000048
:1010700000000000000000002ED0000040B300007F
:10108000447041930A9539F015E11A9521F040B367
:101090004470D9F3E3CFEEE8F1E040814423B9F4A2
:1010A00047814423B1F059D005C0909A0000000058
:1010B000909800C041E0E5EFF1E040837F911F91FF
:1010C0000F914F91FF91EF911FBE1F90189532D055
:1010D000F1CF1DD0EFCF12E01A95F1F708950F93DD
:1010E0001F93442700E81191112309F0402B069526
:1010F000D1F71F910F9108950F931F9300E8142FBC
:10110000102311930695D9F71F910F910895AF936E
:10111000BF93AFEEB1E0EEE8F1E04D91EDDF4D9120
:10112000EBDF4D91E9DFBF91AF91EEE8F1E078E1BF
:1011300021D00895AF93BF93A2EFB1E0EEE8F1E0C4
:101140004D91DADF4D91D8DF4D91D6DFBF91AF9150
:10115000EEE8F1E078E10ED00895E6EFF1E070817D
:10116000772319F4EFEAF1E002C0EFECF1E070E26E
:1011700001D008953F934F937F9331913323E1F44E
:1011800000008A9A44E14A95F1F700008A9844E009
:101190004A95F1F77A9589F70000000000000000F9
:1011A000000000008A9A48E04A95F1F700008A980A
:1011B0007F914F913F9108958A9A46E04A95F1F7C1
:1011C000000000008A9842E14A95F1F70000000013
:1011D0007A9599F600000000000000000000000071
:1011E0008A9A44E04A95F1F700008A987F914F91DE
:1011F0003F910895FC0109C0992787FD90958617B6
:10120000970711F441830895329680818F3FA1F7AB
:101210000895FC018081823011F080E00895818181
:101220000895FC018081833041F0843091F0813059
:1012300011F020E014C0218112C03281818137FF7A
:1012400004C020E038175CF009C020E083173CF0B0
:1012500005C020E09181828189170CF021E0822F66
:101260000895CF92DF92EF92FF920F931F93CF9347
:10127000DF938C017B016A01FA0103C083818183C2
:10128000349680818823D1F73DC0282F332727FD4E
:101290003095F8018181C82FDD27C7FDD095CC0F8F
:1012A000DD1FCC0FDD1FCC0DDD1D8881823081F06C
:1012B0008330D1F0813021F5220F331F220F331FED
:1012C000C701820F931FADDF9981982B998318C0B6
:1012D000F901EE0FFF1FEE0FFF1FEE0DFF1D8081C6
:1012E000823071F481810BC0220F331F220F331F14
:1012F000C701820F931F95DF882311F08A818983AC
:101300000E5F1F4FF80180818F3F09F0BECFDF9144
:10131000CF911F910F91FF90EF90DF90CF900895A4
:10132000C198B99A0895892B11F41FBC089581E8DA
:101330008FBD8AE08EBD1BBC8FE18ABD08950F93DF
:101340001F93CF93DF93EC0100E911E081E090E07F
:10135000EADF80EB94E0F8013197F1F70197D9F7D4
:1013600080E090E0E0DF84EF91E0F8013197F1F761
:101370000197D9F7219751F7DF91CF911F910F91E5
:1013800008951F920F920FB60F9211248F938091A0
:10139000F7018C3318F48F5F8093F7018F910F90D2
:1013A0000FBE0F901F90189589B78E7F89BF089543
:1013B00089B7816089BF089585E083BF12BE89B770
:1013C000816089BF1092F70108958091F7018C33F5
:1013D00010F480E008951092F70181E008958EE303
:1013E00092E060E070E049E051E01AD208958EE3A7
:1013F00092E060E070E049E051E002D28EE392E0DA
:101400006EE671E047E050E0E7D1009719F420E084
:1014100030E01DC0AEE3B2E0EEE6F1E087E001901F
:101420000D928150E1F7109245021092460287E436
:1014300092E06FEF70E040E051E0DBD18EE392E0AC
:1014400060E070E049E051E0EBD121E030E0C9011B
:1014500008951FBC83E08EBD1DBC1CBC1092FA0118
:1014600086ED96E09093F9018093F801089508B60F
:1014700002FE0AC088B7846088BF86ED96E090932C
:10148000F9018093F8013EC08CB59DB523E0893EFB
:10149000920710F126E0873D920718F08E5E924089
:1014A00002C086ED96E09093F9018093F801809157
:1014B000F8019091F901885E934030F486ED96E052
:1014C0009093F9018093F8011092FB011DBC1CBCA4
:1014D00088B7846088BF14C08091FB018F5F8093C0
:1014E000FB01893078F01DBC1CBC88B7846088BFC4
:1014F00081E090E09093F9018093F8011092FB0154
:101500001092FA011DBC1CBC88B7846088BF109281
:10151000FA0108958091FA01882369F42CB53DB54C
:101520008091F8019091F9012817390720F081E0A6
:101530008093FA01089580E00895A398AB98BC9A2F
:10154000C4980895EF92FF920F931F93CF93DF9368
:101550007C01662309F456C070E020E030E0E0E052
:10156000F0E011C088818423FD01E95BFC4F80839A
:1015700011964695A017B107A9F72F5F3F4F261781
:10158000370754F4FD01DF0140E8E701C20FD31F24
:101590008F01085F1F4FE6CFE7E4F3E0CF93DF93BF
:1015A000EF93FF930191002311F069F41BC0000039
:1015B000A39A1DE014D0A3980000000000000000D2
:1015C000119781F70FC0A39A12E0000008D0A398EA
:1015D00019E005D000000000119721F703C01A950B
:1015E000F1F7089500000000FF91EF91DF91CF9196
:1015F000A39A12E00000F3DFA3980FEF0A9511F011
:101600009B9BFCCFE7E4F3E0EF93FF9311270027C8
:101610000395A1F09B99FCCF08C00BE4039572F0F1
:101620009B99FCCF139551F001930BE4039532F095
:101630009B9BFCCF139511F00193EFCFFF91EF919E
:10164000612F70E06115710531F110FF24C040E099
:1016500050E020E030E00CC08081F901EA5BFC4FF3
:101660009081E0E0891708F4E1E0EC934F5F5F4F71
:10167000DA01A95BBC4FF901E95BFC4F2E5F3F4FDC
:10168000411750F38AE18A95F1F79B0121503040D0
:101690003595279502C020E030E0C901DF91CF9158
:1016A0001F910F91FF90EF900895DF93CF930F92CA
:1016B000CDB7DEB71982CE01019661E070E042DF5E
:1016C000009719F420E030E026C0489711F580918A
:1016D0004B03882311F098E001C090E080914C0307
:1016E0008111946080914D038111926080914E032D
:1016F000811191609A3028F4983028F4953049F49B
:1017000005C09B3031F422E030E005C021E030E03C
:1017100002C023E030E0C9010F90CF91DF9108951E
:10172000629FD001739FF001829FE00DF11D649FC5
:10173000E00DF11D929FF00D839FF00D749FF00D51
:10174000659FF00D9927729FB00DE11DF91F639FF2
:10175000B00DE11DF91FBD01CF011124089597FBC4
:10176000092E05260ED057FD04D014D00AD0001C37
:1017700038F450954095309521953F4F4F4F5F4F2E
:101780000895F6F790958095709561957F4F8F4FEE
:101790009F4F0895A1E21A2EAA1BBB1BFD010DC08D
:1017A000AA1FBB1FEE1FFF1FA217B307E407F50711
:1017B00020F0A21BB30BE40BF50B661F771F881FED
:1017C000991F1A9469F760957095809590959B0183
:1017D000AC01BD01CF010895FB01DC0104C08D9176
:1017E0000190801921F441505040C8F7881B990B93
:1017F0000895DC0101C06D9341505040E0F7089519
:10180000DC01CB01FC01E199FECF06C0FFBBEEBBC2
:10181000E09A31960DB20D9241505040B8F70895BC
:10182000DC01CB0102C02D9105D041505040D8F7CA
:101830000895262FE199FECF9FBB8EBB2DBB0FB61F
:10184000F894E29AE19A0FBE01960895F894FFCFBA
:101850000000010102020303040405050606070750
:10186000080809090A0A0B0B0C0C0D0D0E0E0F0FC0
:10187000101411141214131414141514161417142C
:10188000181419141A14FFFF0800000000000000CB
:1018900000001808E107B906A506100801000100BC
:1018A0000000010000000100000001000000010034
:1018B0000000010000000300E0000300200003001E
:1018C000E000030020000100000001000000010012
:1018D0000000010000000200000002000000010002
:1018E0000000010000000300E000030020000300EE
:1018F000E00003002000040020000400200002009B
:1019000000000200000000000000010000000100D3
:1019100000000100000001000000010000000100C3
:1019200000000100000001000000010000000100B3
:1019300000000100000001000000010000000100A3
:10194000000002000000020000000300810003000C
:101950007F000300810003007F0000000000474378
:08196000324E363476350000EA
:00000001FF
